:03000000020008F3
:0300610002000397
:0500030012006480FE04
:100064007A2D7B0BEAB503028015C3EB9A5008EA9C
:10007400C39BFA8A8080EDEBC39AFB8B9080E5BA30
:10008400010BBB010875A0AA75B0AA800675A0551E
:0500940075B00180FEC3
:06003700E478FFF6D8FD9D
:100015007900E94400601B7A0090009D780075A086
:1000250000E493F2A308B8000205A0D9F4DAF2754A
:02003500A0FF2A
:10003D007800E84400600A790075A000E4F309D85F
:10004D00FC7800E84400600C7900900000E4F0A317
:04005D00D8FCD9FAF8
:0D000800758107120099E582600302000374
:04009900758200224A
:00000001FF
